:020000040800F2
:10000000D00500202902000831190008BB1800089B
:100010002D190008BD04000855200008000000004C
:10002000000000000000000000000000351900087A
:10003000C104000800000000331900083719000847
:100040004D0200084D0200084D0200084D02000854
:100050004D0200084D0200084D0200084D02000844
:100060004D0200084D0200084D0200084D02000834
:100070004D0200084D0200084D0200084D02000824
:100080004D0200084D0200084D0200084D02000814
:100090004D0200084D0200084D0200084D02000804
:1000A0004D0200084D0200084D0200084D020008F4
:1000B0004D0200084D0200084D0200084D020008E4
:1000C0004D0200084D0200084D0200084D020008D4
:1000D0004D0200084D0200084D02000805200008EE
:1000E0004D0200084D0200084D0200084D020008B4
:1000F0004D0200084D0200084D0200084D020008A4
:100100004D0200084D0200084D0200084D02000893
:100110004D0200084D0200084D0200084D02000883
:100120004D0200084D0200084D0200084D02000873
:100130004D0200084D0200084D0200084D02000863
:100140004D0200084D0200084D0200084D02000853
:100150004D0200084D0200084D0200084D02000843
:100160004D0200084D0200084D0200084D02000833
:100170004D0200084D0200084D020008000000007A
:100180004D0200084D02000800F002F800F03CF8B3
:100190000AA090E8000C82448344AAF10107DA45E2
:1001A00001D100F031F8AFF2090EBAE80F0013F0F8
:1001B000010F18BFFB1A43F001031847B4210000D8
:1001C000D4210000103A24BF78C878C1FAD8520769
:1001D00024BF30C830C144BF04680C6070470000C1
:1001E0000023002400250026103A28BF78C1FBD840
:1001F000520728BF30C148BF0B6070471FB502F0DF
:10020000A5F81FBD10B510BD00F012F91146FFF79B
:10021000F5FF01F0E5FF00F044F903B4FFF7F2FF4A
:1002200003BC01F035FF00000C48016841F4700187
:1002300001600B4880470B480047FEE7FEE7FEE7FA
:10024000FEE7FEE7FEE7FEE7FEE7FEE7FEE700006B
:1002500005480649044A064B7047000088ED00E057
:100260004119000889010008D0010020D0050020B4
:10027000D0010020704753EA020C00F069802DE99C
:10028000F04B4FF00006002B1FBFB3FA83F503FAC3
:1002900005F424FA05F65E4012BF1643B2FA82F561
:1002A00002FA05F4C5F120051EBF22FA05FC44EA56
:1002B0000C04203556EA044C4FEA144418BF641C61
:1002C0004FF000084FF00009904271EB030C39D356
:1002D000002919BFB1FA81F701FA07F6B0FA80F7E1
:1002E00000FA07F6C7F120071EBF20FA07FC46EA0E
:1002F0000C062037B6FBF4FCA7EB0507103F07F010
:100300001F0BCBF120060CFA0BFB2CFA06F644BFB0
:10031000B3460026202FA4BF5E464FF0000B5BEAD9
:10032000060C08BF4FF0010B19EB0B09ABFB027C6D
:1003300048EB0608C01B06FB02CC0BFB03CC71EBA1
:100340000C01C1E70B46024641464846BDE8F08B2A
:1003500013B54FF000004FF00001AFF30080BDE88F
:100360001C4070470FB4044910B503AA029800F06E
:1003700031F810BC5DF814FB080000204FF00002BB
:1003800000B5134694469646203922BFA0E80C508B
:10039000A0E80C50B1F12001BFF4F7AF090728BF66
:1003A000A0E80C5048BF0CC05DF804EB890028BFE2
:1003B00040F8042B08BF704748BF20F8022B11F00B
:1003C000804F18BF00F8012B704770477047704787
:1003D00070470000074B70B50D467B4400F011F8E4
:1003E0000446284600F020F810B14FF0FF3070BDF1
:1003F000204670BD4B1D000001694A1C026108784F
:10040000704700B58FB0CDE9013100210591054954
:100410007944CDE903101146684600F02EF80FB07C
:1004200000BD0000E5FFFFFF007B00F0800070478B
:10043000754600F03FF8AE4605006946534620F089
:100440000700854618B020B5FFF702FFBDE8204041
:100450004FF000064FF000074FF000084FF0000B80
:1004600021F00701AC46ACE8C009ACE8C009ACE833
:10047000C009ACE8C0098D4670472DE9F041064639
:100480000024D6E90170F5688046304603E0414615
:10049000B847641C3046A8470028F8D12046BDE87C
:1004A000F08110B50446AFF300802046BDE810404F
:1004B000FFF7B3BE004870477001002000BFFEE7A1
:1004C000704770B50446A56D00F072F9064694F8C1
:1004D0003500022808D08020606500BF002084F825
:1004E000340000BF012070BD2068006820F01600B5
:1004F000216808602068406920F080002168486118
:10050000206C08B9A06C28B12068006820F00800B1
:10051000216808602068006820F0010021680860F8
:100520000FE000F045F9801B05280AD920206065FE
:1005300000BF002084F8340000BF032084F8350099
:10054000D1E72068006800F001000028E9D194F8A4
:100550005C103F208840A86000BF002084F8340071
:1005600000BF012084F835000020BCE7014691F867
:100570003500022803D080204865012070470520FF
:1005800081F835000868006820F001000A681060F2
:100590000020F3E7F8B502460B46002500240020B2
:1005A0000021DEE0012606FA01F51E6806EA0504D0
:1005B000AC4275D11E7906F00306012E04D01E79D7
:1005C00006F00306022E13D190684F000326BE40AA
:1005D000B0434F00DE68BE40304390605068012653
:1005E0008E40B0431E79C6F300168E4030435060F3
:1005F0001E7906F00306032E09D0D0684F000326AB
:10060000BE40B0434F009E68BE403043D0601E796C
:1006100006F00306022E13D1CF0802F1200656F889
:1006200027004E07F70E0F26BE40B0434F07FF0EC0
:100630001E69BE403043CF0802F1200646F827006D
:1006400010684F000326BE40B0431E7906F0030633
:100650004F00BE40304310605E6806F08056B6F131
:10066000805F7DD100BF00260096404E366846F47C
:1006700080463E4F3E603E46366806F48046009611
:1006800000BF00BF3A4E8F0856F827008E07370F7D
:100690000F26BE40B043374EB24202D1002624E0BE
:1006A0005EE0354EB24201D101261EE0334EB24229
:1006B00001D1022619E0324EB24201D1032614E0E4
:1006C000304EB24201D104260FE02F4EB24201D18A
:1006D00005260AE02D4EB24201D1062605E02C4E39
:1006E000B24201D1072600E008268F073F0FBE4027
:1006F00030431F4E8F0846F82700264E3068A0432F
:100700005E6806F48036B6F5803F00D12043214E66
:100710003060361D3068A0435E6806F40036B6F5DA
:10072000003F00D120431B4E361D3060361D30681F
:10073000A0435E6806F48016B6F5801F00D1204302
:10074000144E08363060361D3068A0435E6806F4EB
:100750000016B6F5001F00D120430E4E0C36306057
:10076000491C1029FFF41EAFF8BD000044380240B8
:100770000838014000000240000402400008024026
:10078000000C024000100240001402400018024019
:10079000001C0240003C01400AB1816101E00B04F1
:1007A0008361704701480068000C7047002004E036
:1007B00001480068704700001000002003480068EE
:1007C0000349097808440149086070471000002077
:1007D0001800002010B50A48006840F4007008496D
:1007E00008600846006840F480600860032000F05C
:1007F0007FF80F2000F006F800F02AF8002010BD66
:10080000003C024070B504460E4800784FF47A71FF
:10081000B1FBF0F00C490968B1FBF0F5284600F097
:100820001DFC08B1012070BD102C07D2002221460A
:10083000501E00F01EF80548046001E00120F2E7B8
:100840000020F0E718000020000000201400002025
:10085000704701460846002809DB00F01F0301220B
:100860009A4043099B0003F1E023C3F8002100BF35
:1008700070472DE9F05F80460D461646002701F0CF
:10088000EBFB074639462A46334601F00700C0F124
:10089000070ABAF1040F02D94FF0040A01E0C0F1CF
:1008A000070AD14600F1040ABAF1070F02D24FF04D
:1008B000000A01E0A0F1030AD4464FF0010A0AFA47
:1008C00009FAAAF1010A0AEA020A0AFA0CFA4FF036
:1008D000010B0BFA0CFBABF1010B0BEA030B4AEA21
:1008E0000B042146404601F0BFFBBDE8F09F00002D
:1008F00000BF00F00702064B19684FF6FF031940CE
:10090000044B0B4343EA0221014B196000BF7047BF
:100910000CED00E00000FA0570B504460D460CB978
:10092000012070BD5848006800F00700A84209D2B5
:1009300055490D700846006800F00700A84201D034
:100940000120EEE7207800F0020002281DD1207877
:1009500000F00400042805D14C48006840F4E05041
:100960004A490860207800F00800082805D1474867
:10097000006840F46040454908604448006820F041
:10098000F000A168084341490860207800F00100A8
:10099000A8B36068012807D13C4808380068C0F354
:1009A0004040B8B90120BCE76068022802D0606806
:1009B000032807D1354808380068C0F3406048B9BB
:1009C0000120AEE7314808380068C0F3400008B99C
:1009D0000120A6E72D48006820F003006168084365
:1009E0002A490860FFF7E4FE064609E0FFF7E0FE4B
:1009F000801B41F28831884202D9032091E707E049
:100A00002248006800F00C006168B0EB810FEDD166
:100A10001D48006800F00700A84209D91A490D7066
:100A20000846006800F00700A84201D0012078E7DE
:100A3000207800F00400042807D11448006820F44E
:100A4000E050E168084311490860207800F0080090
:100A5000082808D10D48006820F46040216940EA68
:100A6000C1000A49086000F03FF808490968C1F36D
:100A70000311074A515CC8400649086006480068EF
:100A8000FFF7C0FE00204CE7003C0240083802405F
:100A900056230008000000201400002001480068D0
:100AA000704700000000002000B5FFF7F7FF044981
:100AB0000968C1F38221034A515CC84000BD0000AF
:100AC000083802406623000800B5FFF7E7FF044935
:100AD0000968C1F34231034A515CC84000BD0000BF
:100AE00008380240662300082DE9F047002400255D
:100AF0000026A1462548006800F00C0020B104281B
:100B000005D008283AD105E0DFF8849039E0DFF815
:100B1000849036E01D48001F006800F03F041B4829
:100B2000001F006800F4800078B11A481749091FB7
:100B30000968C1F38811A0FB017001462246002319
:100B40003846FFF798FB05460EE011480F49091F8C
:100B50000968C1F38811A0FB0170014622460023F9
:100B60003846FFF788FB05460848001F0068C0F3B9
:100B70000140401C4600B5FBF6F902E0DFF810909A
:100B800000BF00BF4846BDE8F087000008380240BB
:100B90000024F40000127A00F8B504460CB90120D4
:100BA000F8BD207800F00100002874D0F9480068F2
:100BB00000F00C0004280DD0F648006800F00C008E
:100BC000082813D1F348001F006800F48000B0F536
:100BD000800F0BD1EF4808380068C0F34040002870
:100BE00059D06068002856D10120D9E700BF60685D
:100BF000B0F5803F08D1E7480838006840F48030FD
:100C0000E449083908601EE06068B0F5A02F0DD1F6
:100C1000E0480838006840F48020DE490839086060
:100C20000846006840F4803008600CE0D948083875
:100C3000006820F48030D749083908600846006809
:100C400020F48020086000BF606890B1FFF7B0FD1D
:100C5000054606E0FFF7ACFD401B642801D90320E0
:100C60009EE7CC4808380068C0F340400028F1D027
:100C700011E0FFF79DFD054606E0FFF799FD401BDB
:100C8000642801D903208BE7C24808380068C0F304
:100C900040400028F1D1207800F0020002285FD106
:100CA000BC48006800F00C0058B1BA48006800F079
:100CB0000C0008281CD1B748001F006800F4800011
:100CC000B0B9B44808380068C0F3400020B1E0680B
:100CD000012801D0012063E7AE480838006820F001
:100CE000F800216940EAC100AA490839086037E0E4
:100CF000E06800B30120A8490860FFF759FD0546E8
:100D000006E0FFF755FD401B022801D9032047E705
:100D1000A04808380068C0F340000028F1D09D4882
:100D20000838006820F0F800216940EAC1009949BC
:100D30000839086014E0002097490860FFF738FD83
:100D4000054606E0FFF734FD401B022801D90320C9
:100D500026E7904808380068C0F340000028F1D129
:100D6000207800F0080008282CD16069A8B1012083
:100D70008A490860FFF71CFD054606E0FFF718FDED
:100D8000401B022801D903200AE782486C30006822
:100D9000C0F340000028F1D014E000207F49086033
:100DA000FFF706FD054606E0FFF702FD401B02289F
:100DB00001D90320F4E677486C300068C0F34000A6
:100DC0000028F1D1207800F00400042870D1002719
:100DD00070483830006800F0805090B900BF0020A3
:100DE00000906C483830006840F0805069493831D4
:100DF00008600846006800F08050009000BF00BF07
:100E000001276748006800F48070B0B96448006842
:100E100040F4807062490860FFF7CAFC054606E0AE
:100E2000FFF7C6FC401B022801D90320B8E65C4846
:100E3000006800F480700028F2D000BFA06801288C
:100E400008D154486830006840F0010051496831C9
:100E500008601DE0A06805280DD14E486830006884
:100E600040F004004B49683108600846006840F0D3
:100E7000010008600CE047486830006820F001007D
:100E80004449683108600846006820F004000860A2
:100E900000BFA068A8B1FFF78BFC054609E0FFF78B
:100EA00087FC401B41F28831884202D9032077E653
:100EB00026E0384868300068C0F340000028EED0D3
:100EC00013E0FFF775FC054608E0FFF771FC401BD7
:100ED00041F28831884201D9032061E62D4868300B
:100EE0000068C0F340000028EFD1012F07D1294846
:100EF0003830006820F0805026493831086000BF43
:100F0000A069002845D02348006800F00C0008289C
:100F10005DD0A069022845D100201F490866FFF76F
:100F200047FC054606E0FFF743FC401B022801D9B9
:100F3000032035E6174808380068C0F340600028F1
:100F4000F1D1D4E907010843616A40EA8111012225
:100F5000A06AC2EB500041EA00412C20005D41EA4A
:100F600000600C49091F086001200B490866FFF763
:100F70001FFC054606E0FFF71BFC401B022801D9B9
:100F800003200DE6034808380068C0F340600028DD
:100F9000F1D049E00838024000004742800E474245
:100FA00000700040002021490866FFF701FC05465B
:100FB00006E0FFF7FDFB401B022801D90320EFE507
:100FC0001B480068C0F340600028F2D12CE0A06903
:100FD000012800D1E4E51648001D0668A069012833
:100FE00020D006F48001E06981421BD106F03F0168
:100FF000206A814216D147F6C0703040616AB0EB7A
:10100000811F0FD106F440310122A06AC2EB5000CB
:10101000B1EB004F06D106F070612C20005DB1EB02
:10102000006F01D00120BBE50020B9E50000474278
:1010300000380240042808D14FF0E021096941F04E
:1010400004014FF0E022116107E04FF0E02109694F
:1010500021F004014FF0E0221161704770B50446A1
:101060002546681EB0F1807F01D301200FE0681E85
:101070004FF0E02148610F214FF0FF3000F0F4FF06
:1010800000204FF0E021886107200861002070BD3A
:1010900030B502460B4600BF92F83C00012801D152
:1010A000022030BD012082F83C0000BF022082F8FF
:1010B0003D00106844681068816824F07004186866
:1010C000044310684460184D1068A8421BD0106893
:1010D000B0F1804F17D0154D1068A84213D0144DB1
:1010E0001068A8420FD0134D1068A8420BD0124DC3
:1010F0001068A84207D0114D1068A84203D0104DC7
:101100001068A84205D121F0800158680143106899
:101110008160012082F83D0000BF002082F83C0081
:1011200000BF00BFBDE70000000001400004004018
:1011300000080040000C0040000401400040014055
:101140000018004010B586B00446142101A8FFF72E
:1011500015F92068B0F1804F1BD100BF002000902E
:101160000D48006840F001000B490860084600681F
:1011700000F00100009000BF00BF0220019002902B
:101180000020039004900120059001A90348FFF777
:1011900001FA06B010BD00003038024000000240E5
:1011A00070B504460D46164600BF94F83C00012871
:1011B00001D1022070BD012084F83C0000BF36B18F
:1011C000042E1BD0082E31D00C2E5ED145E02946CE
:1011D000206800F03DFC2068806940F0080021682C
:1011E00088612068806920F0040021688861206897
:1011F0008069296908432168886147E02946206899
:1012000000F05EFC2068806940F40060216888611D
:101210002068806920F48060216888612068806986
:10122000296940EA0120216888612FE02946206869
:1012300000F084FC2068C06940F008002168C861A3
:101240002068C06920F004002168C8612068C06976
:10125000296908432168C86118E02946206800F020
:10126000A9FC2068C06940F400602168C86120685A
:10127000C06920F480602168C8612068C06929695C
:1012800040EA01202168C86100E000BF00BF00BF44
:10129000002084F83C0000BF00BF8BE710B5044677
:1012A0000CB9012010BD94F83D0028B9002084F845
:1012B0003C00204600F026F8022084F83D00211D65
:1012C000206800F047FB012084F8460000BF84F846
:1012D0003E0001213F20015540200155412001558C
:1012E00000BF00BF012084F8420043200155442084
:1012F00001554520015500BF012084F83D00002024
:10130000D0E7000008B50168B1F1804F0FD100BFF0
:10131000002100910649096841F00101044A116069
:101320001146096801F00101009100BF00BF08BD2E
:101330004038024070B504460D4615B994F83E0099
:101340000BE0042D02D13F20005D06E0082D02D104
:101350004020005D01E04120005D012801D0012016
:1013600070BD1DB9022084F83E000EE0042D03D1AB
:1013700002213F20015508E0082D03D10221402021
:10138000015502E002214120015501222946206831
:1013900000F04CFB23492068884203D02249206892
:1013A000884201D1012000E0002028B12068406C73
:1013B00040F40040216848641A49206888421BD0E4
:1013C0002068B0F1804F17D018492068884213D0A8
:1013D0001749206888420FD01649206888420BD0F0
:1013E00011492068884207D013492068884203D0F9
:1013F0001249206888420CD12068806800F00706F6
:10140000062E0CD02068006840F0010021680860BA
:1014100005E02068006840F00100216808600020B5
:101420009EE700000000014000040140000400406D
:1014300000080040000C004000400140001800403F
:101440007047704701460022002391F83D2091F833
:101450003E3042EA030070472DE9F84F0446206809
:1014600005682068C668206847694FF00009CA46C9
:1014700005F00F09B9F1000F0AD105F0200038B1CD
:1014800006F0200020B1204600F0F3FBBDE8F88F05
:10149000B9F1000F72D007F0010018B906F490708E
:1014A00000286BD005F0010030B106F4807018B14F
:1014B000206C40F00100206405F0040030B107F01A
:1014C000010018B1206C40F00200206405F0020019
:1014D00030B107F0010018B1206C40F00400206426
:1014E00005F0080048B106F0200010B907F001002F
:1014F00018B1206C40F008002064206C70B305F037
:10150000200028B106F0200010B1204600F0B1FB09
:1015100020684069C0F3801A206C00F0080010B900
:10152000BAF1000F23D0204600F078FB2068406914
:1015300000F04000402816D12068406920F04000AB
:1015400021684861A06B50B15648A16B0865A06B3B
:10155000FFF70CF810B1A06B016D88470CE0204636
:10156000FFF76FFF08E02046FFF76BFF04E020461F
:10157000FFF767FF0020206488E7FFE7206B012862
:1015800079D105F01000002875D006F01000002871
:1015900071D000BF00200090206800680090206893
:1015A0004068009000BF00BF2068406900F0400024
:1015B000402839D1A06B006840681FFA80F8B8F164
:1015C000000F30D0A08D40452DDDA4F82E80A06BFB
:1015D000C069B0F5807F1FD02068C06820F480709B
:1015E0002168C8602068406920F0010021684861D6
:1015F0002068406920F0400021684861202084F87C
:101600003E00002020632068C06820F010002168A0
:10161000C860A06BFEF755FFA08DE28D801A81B2E5
:101620002046FFF70DFF31E7A08DE18D401A1FFA2C
:1016300080F8E08DE8B1B8F1000F1AD02068C068DA
:1016400020F490702168C8602068406920F0010093
:1016500021684861202084F83E0000202063206833
:10166000C06820F010002168C86041462046FFF79E
:10167000E7FE0BE7FFE705F0800030B106F08000E1
:1016800018B1204600F08DFC00E705F0400030B1B5
:1016900006F0400018B1204600F0DBFAF6E600BF85
:1016A000F4E60000091C000810B504460CB901203E
:1016B00010BDA06900B100E000BF94F83D0028B95A
:1016C000002084F83C00204600F028F8242084F80C
:1016D0003D002068C06820F400502168C8602046A2
:1016E00000F026FB2068006920F490402168086122
:1016F0002068406920F02A00216848612068C0689D
:1017000040F400502168C86000202064202084F844
:101710003D0084F83E000020CAE7000010B586B006
:1017200004462E492068884255D100BF00BF0020E2
:1017300000902B48006840F4802029490860084642
:10174000006800F48020009000BF00BF00BF00BF11
:1017500000BF0020009022481038006840F00800C8
:101760001F49103908600846006800F00800009022
:1017700000BF00BF00BF00BF00BF002000900846B0
:10178000006840F0020008600846006800F00200AF
:10179000009000BF00BF00BF88150190022002909A
:1017A00001200390022004900720059001A90D4814
:1017B000FEF7F0FE4FF4006001900720059001A9AC
:1017C0000948FEF7E7FE2720FFF743F803221146FA
:1017D0002720FFF74EF806B010BD0000004800407B
:1017E00040380240000C02400004024070B504463C
:1017F0000D46164694F83E00202816D105B10EB9C4
:10180000012070BD00BF94F83C00012801D10220E6
:10181000F7E7012084F83C0000BF00202063324637
:101820002946204600F09AFBEBE70220E9E700009A
:101830001D4A0168914236D11C49098801F40041D2
:1018400089BB1A49098801F4804171B118490978A6
:101850000A2903D00021154A118024E01349098880
:1018600041F40041114A11801DE0114909780D2908
:1018700006D10E49098841F480410C4A118012E0DA
:101880000B490978094A1288C2F30D02094B995491
:1018900006490988491C054A118011460988C7294B
:1018A00001DD002111807047004800400C0000203D
:1018B0000E0000201C000020704700BFFEE7000063
:1018C00000B589B00020079008901C216846FEF7FB
:1018D00055FD4FF0804014490860532048600021B6
:1018E000114881606321C160002101618161FFF7BE
:1018F000D5FC00200790089007A90B48FFF7C8FB0C
:10190000602000900020019002900490042269461B
:101910000548FFF745FC0448FFF714FC0421024882
:10192000FFF708FD09B000BD2801002000BFFEE759
:1019300070477047704710B5FEF740FF10BD0000BC
:101940000348006840F470000149086070470000D7
:1019500088ED00E010B50268294B98420ED0B0F136
:10196000804F0BD0274B984208D0274B984205D088
:10197000264B984202D0264B984203D122F07002A7
:101980004B681A431E4B984220D0B0F1804F1DD0B7
:101990001C4B98421AD01C4B984217D01B4B9842B4
:1019A00014D01B4B984211D01A4B98420ED01A4BB0
:1019B00098420BD0194B984208D0194B984205D049
:1019C000184B984202D0184B984203D122F440722F
:1019D000CB681A4322F080034C6943EA0402026098
:1019E0008B68C3620B688362054B984202D0084B38
:1019F000984201D10B6903630123436110BD0000CC
:101A0000000001400004004000080040000C0040BD
:101A100000040140004001400044014000480140F2
:101A200000180040001C00400020004030B501F0CC
:101A30001F05012404FA05F3046A9C430462046A46
:101A400001F01F0502FA05F52C43046230BD0000C9
:101A500030B5056A25F001050562026A43688469AC
:101A600024F0700424F003040D682C4322F00202D9
:101A70008D682A43104DA84200D103E00F4DA842C3
:101A800006D100BF22F00802CD682A4322F00402EA
:101A9000094DA84202D0094DA84207D123F4807312
:101AA00023F400734D692B438D692B43436084619C
:101AB0004D684563026230BD0000014000040140F2
:101AC00030B5056A25F010050562026A436884692D
:101AD00024F4E04424F440740D6844EA052422F020
:101AE00020028D6842EA0512124DA84200D103E09F
:101AF000114DA84207D100BF22F08002CD6842EA12
:101B0000051222F040020B4DA84202D00A4DA84215
:101B100009D123F4806323F400634D6943EA85030C
:101B20008D6943EA8503436084614D688563026281
:101B300030BD0000000001400004014030B5056ADE
:101B400025F480750562026A4368C46924F0700454
:101B500024F003040D682C4322F400728D6842EADD
:101B60000522124DA84200D103E0114DA84207D131
:101B700000BF22F40062CD6842EA052222F48062AE
:101B80000A4DA84202D00A4DA84209D123F480533D
:101B900023F400534D6943EA05138D6943EA0513A5
:101BA0004360C4614D68C563026230BD00000140FE
:101BB0000004014030B5056A25F480550562036ACA
:101BC0004468C26922F4E04222F440720D6842EA9D
:101BD000052223F400538D6843EA0533084DA842DB
:101BE00002D0084DA84204D124F480444D6944EA4F
:101BF00085144460C2614D680564036230BD000015
:101C0000000001400004014070B50546AC6B0020A7
:101C1000E085E0842046FFF714FC70BD0168C968C8
:101C200021F490710268D1600168496921F00101D5
:101C300002685161016B012905D10168C96821F071
:101C400010010268D160202180F83E10002101635C
:101C5000704710B504462068C06820F04000216835
:101C6000C860202084F83D002046FFF725FE0020B4
:101C700010BD70B5044694F83E00222856D1A068E5
:101C8000B0F5805F0CD1206950B90025A66A2068A4
:101C90004068C0F308003080A06A801CA06215E094
:101CA000A56A0026A068B0F5805F03D0A06828B9B7
:101CB000206918B920684068287004E020684068EE
:101CC00000F07F002870A06A401CA062E08D401EDA
:101CD00080B2E08540BB2068C06820F02000216809
:101CE000C8602068C06820F480702168C8602068DF
:101CF000406920F0010021684861202084F83E00FE
:101D0000206B01280AD12068C06820F010002168EB
:101D1000C860A18D2046FFF793FB02E02046FFF745
:101D200087FD0020206370BD0020FCE70220FAE759
:101D30002DE9F84F04462068006920F44050E1681E
:101D40000843216808612169A06808436169084364
:101D5000E169084300902068C06849F20C6188433B
:101D6000009908432168C8602068406920F44070E9
:101D7000A16908432168486176492068884203D0F8
:101D800075492068884203D1FEF79EFE814602E035
:101D9000FEF78AFE8146E069B0F5004F6CD1022063
:101DA0006168A0FB015003461920A9FB00700146A1
:101DB0002A463846FEF75FFA6421B0FBF1F04FEA9D
:101DC000001A02206168A0FB01510B461920A9FBF3
:101DD00000712A463846FEF74EFA834602206168B3
:101DE000A0FB015003461920A9FB00712A46384682
:101DF000FEF741FA6421B0FBF1F000EBC00101EB0A
:101E00000010ABEB8000322101EBC0006421B0FB7D
:101E1000F1F000F0F8000AEB400A02206168A0FB34
:101E2000015003461920A9FB007001462A46384696
:101E3000FEF721FA834602206168A0FB01500346A9
:101E40001920A9FB00712A463846FEF714FA6421CE
:101E5000B0FBF1F000EBC00101EB0010ABEB800038
:101E6000322101EBC0006421B0FBF1F000F007006B
:101E70005044216888606AE004206168A0FB01503A
:101E800003461920A9FB007001462A463846FEF792
:101E9000F2F9824604206168A0FB01500346192034
:101EA000A9FB007001462A463846FEF7E4F9642192
:101EB000B0FBF1F000EBC00101EB0010AAEB8000D9
:101EC000322101EB00106421B0FBF1F000F0F00AC8
:101ED00004206168A0FB017003461920A9FB005192
:101EE0003A462846FEF7C7F96421B0FBF1F00AEB49
:101EF000001A04206168A0FB01510B461920A9FBC0
:101F000000712A463846FEF7B6F983460420616818
:101F1000A0FB015003461920A9FB007001462A4688
:101F20003846FEF7A8F96421B0FBF1F000EBC001E0
:101F300001EB0010ABEB8000322101EB00106421BB
:101F4000B0FBF1F000F00F00504421688860BDE85C
:101F5000F88F0000001001400014014010B5034646
:101F600099629A85DA8500201864222083F83E0061
:101F700000BF002083F83C0000BF1868C06840F430
:101F800080701C68E0601868406940F001001C68BF
:101F900060611868C06840F020001C68E0600020A4
:101FA00010BD014691F83D00212828D18868B0F580
:101FB000805F0BD1086948B90A6A1088C0F308002D
:101FC0000B685860086A801C086205E00B6A581CA0
:101FD000086218780B685860C88C401E80B2C884AC
:101FE00058B90868C06820F080000B68D86008689D
:101FF000C06840F040000B68D860002070470220A5
:10200000FCE7000070B500240F4D1048FFF724FADC
:1020100000BF03E0641CAC4200D904E00B48FFF7AA
:1020200011FA2028F6D100BF002403E0641CAC4262
:1020300000D906E0012206490448FFF7D7FB002833
:10204000F4D100BF70BD0000FFFF0100E4000020DC
:102050000E00002000BFFEE702480068C0F3022027
:10206000704700000CED00E010B5002804DB0A0703
:10207000130E054A135406E00A07140E034A00F033
:102080000F031B1FD45410BD00E400E018ED00E066
:1020900000BF704710B504460420FEF7CBFF01488F
:1020A000046010BD0400002070B504464FF40770B2
:1020B00094FBF0F594FBF0F100FB114603E00748B8
:1020C00000F00EF86D1E002DF9D12EB14FF47A718B
:1020D00006FB01F000F004F870BD0000603D080050
:1020E00070B5034600224FF0E02675690D4E366844
:1020F00003FB06F44FF0E026B16910E04FF0E02654
:10210000B06988420BD0884202D20E1A324402E0F3
:102110002E1A0E4432440146A24200D300E0EDE7FD
:1021200000BF70BD0400002000BF054A126802F025
:102130004002002AF9D0C2B2014B1B1D1A60704741
:102140000048004000B587B000BF00BF00200190EC
:102150002148006840F020001F49086008460068D8
:1021600000F02000019000BF00BF00BF00BF00BF13
:10217000002001900846006840F0200008600846F2
:10218000006800F02000019000BF00BF00BF4815AC
:1021900002900120039004900220059002A90F48AC
:1021A000FEF7F8F94FF48060029002A90B48FEF7A1
:1021B000F1F900BF00224FF400710848FEF7ECFA75
:1021C00000BF00BF00224FF480610448FEF7E4FA2C
:1021D00000BF07B000BD00003038024000140240CC
:1021E00000BF00BFFEF7F6FA0723022208214FF4D2
:1021F000A87000F021F8A820FFF74CFF4FF4E13061
:1022000000F088F8FFF79EFFFFF75AFB05A0FEF7E6
:10221000A9F806E003A0FEF7A5F84FF4FA70FFF75F
:1022200043FFF7E70D0AC4FAB7A2CBCDB5C4CFFB85
:10223000CFA2CEAA3A0D0A002DE9F04192B0804615
:102240000C4615461E460027302106A8FEF796F8D4
:10225000142101A8FEF792F800BF002000902A4840
:10226000006840F08050284908600846006800F087
:102270008050009000BF00BF00BF002000902348A6
:10228000006840F48040214908600846006800F476
:102290008040009000BF00BF01200690000407901E
:1022A00002200C9041050D91CDF83C800E941095C4
:1022B000119606A8FEF770FC07461FB1012012B068
:1022C000BDE8F0810F2001900220029000200390D1
:1022D0004FF4A05004904FF480500590052101A8C0
:1022E000FEF71AFB07460FB10120E8E7FEF75AFA9E
:1022F00041F20101884205D10548006840F4807030
:10230000034908600020DAE74038024000700040CE
:10231000003C024010B5044609480A4908600846D6
:10232000446000218160C160016181610C214161D3
:10233000FFF7BAF9012204490248FFF757FA10BD26
:1023400000480040E40000200E0000204FF04070E4
:10235000E1EE100A704700000000000000000102DA
:10236000030406070809000000000102030400003E
:1023700090230008000000201C000000C401000899
:10238000AC2300081C000020B4050000E001000898
:102390000024F40000000000000000000000000025
:0C23A00000000000100000000100000020
:040000050800018965
:00000001FF
